:03000000020003F8
:03005C0002005F40
:05005F0012026480FEA6
:0E006400AA83E582900000F0A3EAF09000006D
:09007200E0FAA3E0FB7C007D0034
:0E007B00C3EC9AED64808BF063F08095F0503A
:05008900147E337F002E
:05008E001EBEFF011F72
:0B009300EE4F70F70CBC00E00D80DDAC
:01009E00223F
:0E009F00E582900002F09000037480F0C2A38E
:0700AD00D2A1900002E0FA6D
:0E00B400900003E0FB602A53A1FEEB5A6005AA
:0500C20043A1048003CE
:0300C70053A1FB47
:0D00CA00900003E0FBC313FB900003F090D7
:0E00D70000C8C002120064D00243A10180CF15
:0300E500D2A32281
:0E00E800E582900004F09000057480F0C2A143
:0700F600C2A3900004E0FA30
:0E00FD00900005E0FB602A53A1FEEB5A60055F
:05010B0043A104800384
:0301100053A1FBFD
:0D011300900005E0FBC313FB900005F09089
:0E0120000002C002120064D00243A10180CF91
:03012E00D2A32237
:0E013100C2A29003E8120064D2A27582E2120C
:0C013F0000E87582A31200E87582AF1280
:0C014B0000E87582A01200E87582C8125E
:0C01570000E87582221200E87582811217
:0C01630000E875822F1200E875822F1250
:0C016F0000E87582401200E87582B012B2
:0C017B0000E87582101200E87582001286
:0C01870000E87582AF1200E87582A41237
:0801930000E87582A60200E8F5
:0E019B00AA83E58290000AF0A3EAF090000625
:0E01A900E0FAA3E0FB9000157408F0E4A3F068
:0E01B7008A828B83C002C0031203E7E58285B3
:0E01C50083F0D003D00244B0FCADF08C82C0B9
:0E01D30002C0031200E8D003D00290000AE040
:0E01E100FCA3E0FD74F05CFEE4FFC4CEC45449
:0D01EF000F6ECE540FCE6ECE30E30244F002
:0E01FC00FF4306104306108E82C002C003C0EF
:0E020A0004C0051200E8D005D004D003D002D5
:0E02180053040F7D008C82C002C0031200E868
:0E022600D003D00290000C7408F0E4A3F08A1C
:0E023400828B831202CBAA82AB83900008E07B
:0E024200FCA3E0FD4C601A8AF005F07A017B07
:0302500000800625
:06025300EA2AFAEB33FB7E
:0A025900D5F0F78A828B8302009F24
:010263002278
:070264001201317A007B005A
:0E026B00C3EA9480EB6480948050518A048B27
:05027900057E007F007E
:0E027E00C3EE9440EF648094805037900006E9
:0E028C00EEF0A3EFF09000087401F0E4A3F090
:0E029A008C828D83C002C003C004C005C00664
:0E02A800C00712019BD007D006D005D004D0AD
:0A02B60003D0020EBE00C10F80BE8F
:0702C0000ABA00A70B80A49D
:0402C7009000002281
:06003200E478FFF6D8FDA2
:080010007900E94400601B7A4D
:05001800009004FE78D9
:03001D001F75A0AC
:0A00200000E493F2A308B800020503
:08002A00A0D9F4DAF275A0FF81
:0E02CB00AA83E58290000EF0A3EAF090000EE8
:0E02D900E0FAA3E0FB30E709C3E49AFCE49BE3
:0302E700FD800493
:0402EA008A048B05F2
:0E02EE008C028D0390000CE0FCA3E0FD30E7D5
:0A02FC0009C3E49CFEE49DFF8004AA
:040306008C068D07CD
:0D030A00900010EEF0A3EFF08A828B8312BA
:0E0317000339AA82AB8390000EE0FCA3E0FD48
:0E03250030E70CC3E49AFCE49BFD8C828D83D0
:0103330022A7
:050334008A828B832288
:0E033900AA83E582900012F0A3EAF09000146F
:0C034700E4F0900012E0FAA3E0FB7C0060
:0E035300900010E0FDA3E0FE235401FF703780
:0E036100EECD25E0CD33FE900010EDF0A3EEC2
:0E036F00F0900010E0FDA3E0FEC3EA9DEB9EBF
:0E037D005011EEC313CD13CDFE900010EDF025
:05038B00A3EEF0800864
:080390000C900014ECF080BB9E
:05039800900014E0FAE2
:0E039D00900012E0FBA3E0FC900010E0FDA336
:0E03AB00E0FEC3EB9DEC9E400B900012EBC3F6
:0603B9009DF0EC9EA3F094
:0E03BF00900010E0FBA3E0FCC313CB13CBFCBB
:0E03CD00900010EBF0A3ECF08A031AEB70C264
:0C03DB00900012E0FAA3E08A82F5832271
:080038007800E84400600A7939
:030040000075A0A8
:0600430000E4F309D8FC03
:08004900781FE84400600C7907
:0B00510001900000E4F0A3D8FCD9FAF5
:0E03E700AA83E582900017F0A3EAF0900017B9
:0E03F500E0FAA3E0FB30E709C3E49AFCE49BC6
:03040300FD800475
:040406008A048B05D4
:0E040A008C028D03900015E0FCA3E0FD33E4AE
:0D04180033FE6009C3E49CFFE49DF88004FE
:040425008C078D00B3
:0E042900900019EFF0A3E8F08A828B83C006E2
:0E04370012045FAA82AB83D006900017E0FC8F
:0E044500A3E0FD33E4336E600CC3E49AFCE4E4
:070453009BFD8C828D8322CA
:05045A008A828B832261
:0E045F00AA83E58290001BF0A3EAF090001D36
:0E046D00E4F0A3F0900019E0FAA3E0FB7C108D
:0C047B0090001BE0FDA3E0FE339200EEB9
:0E048700CD25E0CD33FE90001BEDF0A3EEF08E
:0E04950090001DE0FDA3E0FECD25E0CD33FE7E
:0C04A30090001DEDF0A3EEF03000129070
:0E04AF00001DE0FDA3E0FE90001D74014DF065
:0304BD00A3EEF0BB
:0E04C00090001DE0FDA3E0FEC3ED9AEE9B4010
:0D04CE001D90001DEDC39AF0EE9BA3F09071
:0E04DB00001BE0FDA3E0FE90001B74014DF03D
:0304E900A3EEF08F
:0E04EC00DC8D90001BE0FAA3E08A82F58322EB
:03000300758120E4
:0A0006001204FAE582600302005FB5
:0404FA0075820022E5
:00000001FF
